:02000000CA290B
:08000800DF00030E8312B400B7
:0E0010000A0EB500040EB6008A110A12F1297C
:1000200000000000CF0B10280800CB08031D192882
:100030000800F9300000000000000000000000008F
:1000400000000000000000000000000000000000B0
:1000500000000000FF3E031D1A2800000000000001
:100060000000000000000000000000000000000090
:10007000000000000000000000000000CB0B192869
:100080000800FA30CB001520FA30CB001520FA30EA
:10009000CB001520FA30CB001520CA0B41280800F0
:1000A0009F185028CB08031969281E08CC00CD01E1
:1000B000CC0DCD0DCC0DCD0DFC30CC0583161E0C1A
:1000C0008312CE00CE0CCE0E03304E05CC04CD08EC
:1000D0006C281E08CC00CD0102301F049F004C0884
:1000E000CE004D08CF00080007304C05CF004F0E62
:1000F000F03983169F0083124B08003A031D8928AC
:100100000130C9000030BA008530B90001308316D3
:1001100091008312390884000008C8004908480487
:10012000CF0080004B08CF00CF0DCF0DFC304F0526
:1001300001389F004D0303191F174E08CF001020F0
:1001400002301F049F000800831239088400480809
:1001500080008316910183129F01080010308312E2
:10016000CA008316071683124A08103A031D0800B6
:1001700010300705CA00B328FF308312CB00831666
:100180000716103083120705CB004B08CC0008007F
:10019000FF308312CB0083168716203083120705A9
:1001A000CB004B08CC0008008316051183120515FF
:1001B00008008316051183120511080083168711A4
:1001C0008312871108008316871183128715080090
:1001D000831607118312071508008316071183126F
:1001E00007110800831687108312871408008316EE
:1001F00087108312871008008316071083120714D4
:100200000800831607108312071008008312CB0121
:100210000330CC00CD012830CE007420CB0150201B
:100220004E08CA00A4204A08CB000800C820CA0112
:10023000CC08031D4A1444104A08031D44144418F2
:1002400008000121D9206430CB001520F720E320DD
:100250006430CB001520F220DE202329BC20CA0107
:10026000CC08031D4A14C4104A08031DC414C41C3E
:10027000080001210A30CB001520D920F720E32007
:10028000C41544110800BC20CA01CC08031D4A143F
:10029000C4104A08031DC414C4180800AE20D4209A
:1002A000DE20C7010A30470203186629F220FF301A
:1002B000CB001520F530CB001520F720FF30CB0008
:1002C0001520F530CB001520C70A52294415F2201D
:1002D00006214B08C60046080A3C03188329012161
:1002E000D920E820F220E320FF30CB0015202D306C
:1002F000CB001520F720DE20FF30CB0015202D305D
:10030000CB0015207129FC20C4110800D92001213F
:10031000F720ED20E320080006214B08C600460820
:100320000A3C0318AD29450AC50045083C3C0318A2
:1003300008000121D920E820F220E320FF30CB0083
:1003400015202D30CB001520F720DE20FF30CB000C
:1003500015202D30CB0015209B29C50108008316E0
:100360009101073083129900C0308316810001305B
:100370008312CA004120C4154410C601C4104411A0
:10038000C5018621C4194321441DC22916218C218F
:100390002E21C229D5308312A000C430A100BB3069
:1003A000A200DC30A300A401A501A601A701A801B9
:1003B000A901AA01AB01AC01AD01AE01AF01BE01C3
:1003C000BF01B701B801C001C101C201C301B00141
:1003D000B101B201B301BC01BD01BB018A110A1216
:1003E000AF298312360E8400350E8A00340E830046
:0603F000DF0E5F0E0900A4
:02400E00420E60
:00000001FF
